:10000000370101002920A9487300000082804EB802
:10001000130101801301018605650A95233485FCCF
:1000200005650A95233025FD05650A95233C45FBAA
:1000300005650A95233865FB08089305F57F9385C8
:10004000157A232005001105E31DB5FE4245D24572
:10005000130645003345A5202E955105B3F5C50E71
:100060003355C50E4D8D0DCD3345A5208545050570
:100070002AC82ECA0DE905650A95033485FC056575
:100080000A95033905FC05650A95033A85FB056564
:100090000A95033B05FB1301017F1301017B4EBE53
:1000A00005452AC82ACA8144930B0101930981029C
:1000B0000949054A254B994A080809A89304E5FF10
:1000C00033C574210C41FD150CC1D5D54C4199C9DE
:1000D000104554452E96B69510C54CC523222501D2
:1000E00091E519A84C452322250199C50946FD151E
:1000F0000506F5FD50C14CC5232C2501232E4501D5
:10010000A90433C574210C4185050CC199C54C4522
:100110002320550131058D04FDF91385D4FF3344A7
:100120007521084009ED1385B4FFB34575218C4155
:10013000B9E969B7032544FF5114F5146DD583253A
:10014000C4FF032684FFB365B5203325C520232CC7
:10015000A4FE232EB4FE2320440113F5F50F7520D1
:10016000032584FF61D98325C4FF0A05898D232CCB
:1001700004FE232EB4FE7DBF7915B3457521904151
:100180007D1690C105DE1505B345752190416DD6EC
:10019000904523A6650109CADD567D16850675FEC4
:1001A000B306D04090C5D4C523A46501130635001D
:1001B000B34576219441638B460199E232851DA0B7
:1001C00003A6C5FF158E050623AEC5FE23A0450177
:1001D00013066500B3453521328503A645FFD115C9
:1001E000751565FE03A6C5FF41DA23AE05FE90C175
:1001F000B3457521904149FE41B785487300000021
:1002000082809148730000008280AD487300000036
:1002100082809308100873000000828093085008C1
:1002200073000000828093087008730000008280D1
:10023000732510C08280732500C0828093086008F7
:100240007300000082800589F322008093920248A7
:10025000B3E2A20073900280828095487300000090
:10026000828093080008730000008280A148730018
:100270000000828093083008730000008280930899
:080280004008730000008280B9
:00000001FF
